:0400000002003F3289
:01000B0032C2
:0100130032BA
:01001B0032B2
:0100230032AA
:01002B0032A2
:01003300329A
:03003B00021C455F
:0300BF000200C27A
:0500C20012017A80FE2E
:0E00C700E582900001F0900001E0FAF582025F
:0200D5001054C5
:0E00D700E582900002F0900002E0FAF582123D
:0E00E50021CAAA82AB83ACF0FDE4C0E074EC4B
:0E00F300C0E07476C0E07446C0E08A828B8361
:0E0101008CF0ED12028DAA82AB83ACF0FDE50E
:0E010F008124FCF581E4C0E0C0E074FAC0E099
:0E011D007443C0E08A828B838CF0ED120CFBE1
:0E012B00AA82AB83ACF0FDE58124FCF581E4F3
:0E013900C0E0C0E0747AC0E07444C0E08A8286
:0E0147008B838CF0ED121D37AA82AB83ACF0D7
:0E015500FDE58124FCF5818A828B838CF0ED20
:0E0163001210FDAA82AB83900003740AF0E430
:09017100A3F08A828B830201BF16
:07017A001221A51203E1129E
:09018100102A12025A75820212C2
:02018A0003F878
:0C018C001210D47582021203F9AA82122C
:0C01980000D7AA82AB83C002C0037437FA
:0B01A400C0E07423C0E07480C0E012D3
:0E01AF001271E58124FBF58190012C12025D96
:0201BD0080CDF3
:0C23370025642064656772656520430022
:0E01BF00AA83E582900005F0A3EAF090000705
:0E01CD00E4F0A3F0900003E0FAA3E0FB7C1046
:0C01DB00900005E0FDA3E0FE339200EE72
:0E01E700CD25E0CD33FE900005EDF0A3EEF047
:0E01F500900007E0FDA3E0FECD25E0CD33FE37
:0C020300900007EDF0A3EEF03000129028
:0E020F000007E0FDA3E0FE90000774014DF033
:03021D00A3EEF05D
:0E022000900007E0FDA3E0FEC3ED9AEE9B40C8
:0D022E001D900007EDC39AF0EE9BA3F09029
:0E023B000005E0FDA3E0FE90000574014DF00B
:03024900A3EEF031
:0E024C00DC8D900005E0FAA3E08A82F58322A3
:03025A0002053961
:0E025D00AA83E582900018F0A3EAF090001842
:0E026B00E0FAA3E0FB900024EAF0A3EBF09091
:08027900000975F00012053FB9
:0C02810090000975F0001205A250F52253
:06028D00120330BC000367
:030293000211F75E
:08029600EF60FA30D502B2D18D
:08029E00E583B4FF0302120D19
:0802A600E582B4FF0302120D12
:0B02AE00258340072482400B0211F75B
:0802B900248314500302120D0E
:0E02C100F582EA8DF0A4A8F0EA8EF0A428F8E9
:0E02CF00E435F0F9EB8DF0A428E935F0F9E400
:0E02DD0033CA8FF0A429F9EA35F0FAEBF88E57
:0E02EB00F0A429F9EA35F0FAE433FBEC8DF0CB
:0E02F900A429F9EA35F0FAE43BFBE88FF0A403
:0E0307002AFAEB35F0FBE433CCFD8EF0A42A8D
:0E031500FAEB35F0FBE43CFCED8FF0A42BFB83
:0A032300EC35F0FC20E70312035E46
:03032D000211D6E4
:0D033000AA82AB83A2F73392D16002D2F70C
:0E033D00F582ACF0E58124F9F8E6FD08E6FE55
:0E034B000886F008E6A2F73392D56002D2F7DA
:05035900F583AFF02266
:06008F00E478FFF6D8FD45
:02035E00780421
:0E036000EC700DC9CACBFCE58224F8F582D8FA
:02036E00F1227A
:020370007820F3
:0E03720020E7111582C3E933F9EA33FAEB33C1
:06038000FBEC33FCD8EC9D
:010386002254
:08004C007909E94400601B7A08
:05005400019023A978D2
:03005900E275A0AD
:0A005C0000E493F2A308B8000205C7
:08006600A0D9F4DAF275A0FF45
:0E0387009000641206161207BEE5828583F010
:0903950090001AF0A3E5F0F0223B
:0D039E0090001AE0FAA3E0FB8A828B831224
:0903AB0007C71207607582901269
:0D03B40007724020758240120772400F90C2
:0C03C100001EE0FAF582120772400302F1
:0203CD00076ABD
:0903CF0012076A758202021BBCD0
:0903D80012076A758201021BBCC8
:0E03E1009000641206161207BEE5828583F0B6
:0903EF0090001CF0A3E5F0F022DF
:0103F80022E2
:0E03F900E58290001FF090001CE0FAA3E0FBEC
:0E0407008A828B831207C712076075829012DB
:0C0415000772402890001FE0FAF58212E8
:0B0421000772402512076075829112DF
:07042C0007724011C201122A
:0E04330007B1AA82C00212076AD0028A822292
:0904410012076A758201121BBC4E
:09044A0012076A758202021BBC54
:0E045300E582900020F0900020E0FAF5821281
:0E04610003F9AA827B008A057C00EA2CFAEBE4
:06046F003D8A82F58322A4
:0E047500AAF0AB83E582900021F0A3EBF0A388
:0E048300EAF090001CE0FAA3E0FB8A828B8373
:0A0491001207C7120760758290126F
:09049B0007725005740124FF22D0
:0D04A4007582041207725005740124FF22B6
:0E04B1001207607582911207725005740124C3
:0204BF00FF221A
:0604C100D2011207B19008
:0C04C7000021E0FAA3E0FBA3E0FC7D00B4
:0E04D300902343E493FEC3ED9E50547F001E21
:0404E100BEFF011F3A
:0E04E5008D007900E8B50608E9B507047E0031
:0204F300800285
:0204F5007E0186
:0C04F700EE24FF9201ED2AFEE43BFF8C96
:0E05030000C002C003C004C005C006C007C08F
:0E051100001207B1A982D000D007D006D00595
:0E051F00D004D003D0028E828F8388F0E912C0
:05052D000CE20D80A1AD
:0705320012076AE424FF2216
:012343000495
:012344000197
:06053900121C710207E82C
:0E053F00AAF0AB83E582900026F0A3EBF0A3B8
:0E054D00EAF0900026E0FAA3E0FBA3E0FC74C5
:09055B000B2AF508E43BF5098CBC
:0C0564000A121C1DAD82AE83AFF0F890AF
:0E0570000024E0F9A3E0FAE4FBFCE92DFDEA2B
:0C057E003EFEEB3FFFEC38F8850882855C
:07058A000983850AF0ED1260
:0A0591000CE2A3EE120CE2A3EF123D
:07059B000CE2A3E8020CE2F0
:0A05A200C00E85810EC082C083C028
:0E05AC00F0E5812407F581121C1DAD82AE839F
:0C05BA00AFF0FAE50E2404F8A60508A630
:0C05C6000608A60708A602A80E08740B81
:0E05D20026FBE40836FC0886028B828C838AA6
:0C05E000F01221AEFBA31221AEFCA3120E
:0905EC0021AEFAA31221AEFDE5D7
:0C05F5000E2404F8C3EB96EC0896EA080C
:0C06010096ED08965006740124FF80035B
:03060D00E424FFE3
:06061000850E81D00E22D0
:0E061600AA83E582900029F0A3EAF0D297D2E1
:0E06240096120D7AE433FABA010890002C7495
:0406320001F080064D
:0606360090002C7402F09C
:0E063C0090002BE4F0900029E0FAA3E0FB7C94
:01064A0000AF
:03064B00BC0700E9
:05064E0040030206EB71
:0E065300EC75F003A4FDFE90234593CEA39317
:0E066100FF90002CE0F87900900003E8F0A371
:0E066F00E9F08E828F83C002C003C004C00574
:0E067D00C000C0011201BFAE82AF83D001D019
:0E068B0000D005D004D003D002C3EA9EEB9F3E
:0A0699004047ED2445FDE43423FE44
:0E06A3008D828E83A3A3E493FFA2E292DFEF89
:0E06B100A2E192D9EF1392D88D828E83E4934A
:0E06BF00FDA3E493FE900003E8F0A3E9F08DA4
:0E06CD00828E831201BFE5828583F0900029A2
:0706DB00F0A3E5F0F0800937
:0906E2000C90002BECF002064B19
:0E06EB0090002BE0FABA0757EA1490002BF0AB
:0C06F90090002BE0FA75F003A42445FAF1
:0C070500E43423FB8A828B83A3A3E493DB
:0E071100FCA2E292DFECA2E192D9EC1392D8A6
:0E071F008A828B83E493FAA3E493FB90002C70
:0E072D00E0FC900003F0A3E4F08A828B8312BC
:0E073B0001BFE5828583F0900029F0A3E5F070
:01074900F0BF
:0E074A00C2DBC2DCC2DDC2DAD2DE900029E0E2
:08075800FAA3E08A82F5832276
:04076000C2DBD2DD49
:0607640030DBFDC2DD22C6
:04076A00D2DCC2DB40
:04076E0020DCFD226C
:0E077200E58290002DF090002DE0F5DAC2DB5C
:0A07800030DBFDAAD9BA1802801977
:05078A00BA20028018F6
:05078F00BA2802800FF2
:05079400BA3002800EE6
:05079900BA40028005DA
:05079E00BA480B8004C5
:0407A300E424FF2229
:0507A700740124FF2293
:0507AC00740124FF228E
:0607B100A20192DAC2DB96
:0707B70030DBFD85DA822230
:0907BE00AAD87B008A828B8322F9
:0E07C700AA83E58290002EF0A3EAF090002EA7
:0E07D500E0FAA3E0FBEA3392DFEAA2E192D958
:0507E300EA1392D82288
:0E234500660206330105E60003C00002A40094
:0723530001900000260004C8
:0200B900C20281
:0407E80030020122B8
:0C07EC009000E2E4F0A3F0A3F0D202229F
:0E07F800AAF0AB83E582900034F0A3EBF0A3EF
:0E080600EAF0900034E0FAA3E0FBA3E0FC8AE5
:0E081400828B838CF0E4120CE274042AFDE463
:0E0822003BFE8C07900030E0F8A3E0F98D82D9
:0E0830008E838FF0E8120CE2A3E9120CE27442
:0E083E00062AFDE43BFE8C07900032E0F8A392
:0E084C00E0F98D828E838FF0E8120CE2A3E9B2
:0B085A00120CE274012AF514E43BF5D7
:04086500158C169048
:0C08690000E2E0F8A3E0F9A3E0FD851434
:09087500828515838516F0E81256
:0A087E000CE2A3E9120CE2A3ED1254
:0E0888000CE29000E2EAF0A3EBF0A3ECF02209
:0E089600AAF0AB83E58290003EF0A3EBF0A346
:0E08A400EAF090003EE0FAA3E0FBA3E0FC8A3D
:0E08B200828B838CF07401120CE274042AFD18
:0E08C000E43BFE8C07900037E0F8A3E0F98DD2
:0E08CE00828E838FF0E8120CE2A3E9120CE296
:0E08DC0074062AFDE43BFE8C07900039E0F81C
:0E08EA00A3E0F98D828E838FF0E8120CE2A35A
:0C08F800E9120CE274082AF514E43BF548
:04090400158C1690A8
:0C090800003BE0F8A3E0F9A3E0FD85143B
:09091400828515838516F0E812B6
:0A091D000CE2A3E9120CE2A3ED12B4
:0A0927000CE274012AF514E43BF51C
:04093100158C16907B
:0C09350000E2E0F8A3E0F9A3E0FD851467
:09094100828515838516F0E81289
:0A094A000CE2A3E9120CE2A3ED1287
:0E0954000CE29000E2EAF0A3EBF0A3ECF0223C
:0E096200AAF0AB83E582900041F0A3EBF0A376
:0E097000EAF0900047E4F0A3F0A3F09000E25C
:0E097E00E0FAA3E0FBA3E0FC900044EAF0A343
:0C098C00EBF0A3ECF0900041E0F514A3A8
:07099800E0F515A3E0F516E0
:0E099F00900044E0FDA3E0FEA3E0FFBD0007D2
:0709AD00BE0004BF0001229F
:0A09B400EDB5140AEEB51506EFB517
:0409BE00160280039A
:0309C200020A37EF
:0E09C500900047E0FCA3E0FBA3E0FABC00308A
:0E09D300BB002DBA002A74012DF8E43EF98F06
:0D09E10002888289838AF01221AEF8A312E9
:0909EE0021AEF9A31221AEFA902A
:0C09F70000E2E8F0A3E9F0A3EAF080348D
:0C0A030074012CF8E43BF90DBD00010E5D
:0E0A0F008D828E838FF01221AEFDA31221AED8
:0E0A1D00FEA31221AEFF888289838AF0ED12BB
:0A0A2B000CE2A3EE120CE2A3EF129E
:020A35000CE2D1
:0E0A3700900044E0FAA3E0FBA3E0FC9000472F
:0D0A4500EAF0A3EBF0A3ECF00ABA00010BFD
:0E0A52008A828B838CF01221AEFAA31221AEA1
:0E0A6000FBA31221AEFC900044EAF0A3EBF0E1
:060A6E00A3ECF002099F59
:0E0A7400AAF0AB83E58290004AF0A3EBF0A35A
:0E0A8200EAF090004AE0FAA3E0FBA3E0FC8A51
:080A9000828B838CF0020962E5
:0E0A98009000E2E0FAA3E0FBA3E0FCBA000845
:060AA600BB0005BC0002CC
:020AAC0080FECA
:050AAE00120AB380FBF9
:0E0AB3009000E2E0FAA3E0FBA3E0FC90004D0F
:080AC100EAF0A3EBF0A3ECF056
:0E0AC90090004DE0FAA3E0FBA3E0FCBA0007AA
:070AD700BB0004BC0001227A
:0E0ADE008A828B838CF01221AEFDBD01028056
:010AEC000306
:030AED00020BB148
:0E0AF00074042AFDE43BFE8C078D828E838FFA
:0E0AFE00F01221AEFDA31221AEFE74082AF5FF
:060B0C000BE43BF50C8C2C
:0A0B12000DC002C003C004850B8271
:070B1C00850C83850DF0122A
:0A0B230021AEFAA31221AEFBA312CB
:0E0B2D0021AEFCC002C003C004C005C00674A7
:0A0B3B004DC0E0740BC0E0C005C01F
:080B4500068A828B838CF022EA
:0C0B4D00D006D005D004D003D0029203E3
:0C0B5900D004D003D002200303020C1DC6
:0E0B650074062AFDE43BFE8C078D828E838F82
:0B0B7300F01221AEFDA31221AEFE85A2
:060B7E000B82850C83854B
:080B84000DF01221AEFFA312D7
:0D0B8C0021AEF8A31221AEF9C005C0067419
:0A0B9900ABC0E0740BC0E0C005C063
:080BA300068F82888389F0228D
:060BAB00D006D005806CAD
:0E0BB10074042AFDE43BFE8C078D828E838F38
:0E0BBF00F01221AEFDA31221AEFEC002C00353
:0B0BCD00C004C005C00674E0C0E07466
:080BD8000BC0E0C005C00622BD
:0D0BE000D006D005D004D003D002E433F5D8
:0A0BED000BE50B602B74062AFAE4F6
:0E0BF7003BFB8A828B838CF01221AEFAA31294
:0C0C050021AEFBC002C0037419C0E074F3
:080C11000CC0E0C002C0032288
:040C1900D003D00232
:0E0C1D0090004DE0FAA3E0FBA3E0FC0ABA0051
:020C2B00010BBB
:0E0C2D008A828B838CF01221AEFAA31221AEC4
:0E0C3B00FBA31221AEFC90004DEAF0A3EBF0FB
:060C4900A3ECF0020AC951
:0E0C4F00AA83E582900050F0A3EAF09000E244
:0E0C5D00E0FAA3E0FBA3E0FC900052EAF0A353
:0D0C6B00EBF0A3ECF0900050E0FAA3E0FBEA
:0E0C7800900052E0FCA3E0FDA3E0FEBC0008EB
:080C8600BD0005BE0002804D17
:0E0C8E0074062CFFE43DF88E018F8288838966
:0E0C9C00F01221AEFFA31221AEF8EFB5020B4D
:0B0CAA00E8B503078C828D838EF022DA
:050CB5000CBC00010D64
:0E0CBA008C828D838EF01221AEFCA31221AE2F
:0E0CC800FDA31221AEFE900052ECF0A3EDF061
:050CD600A3EEF0809D7B
:070CDB0090000075F00022FB
:0323A90000000031
:0E0CE20020F71030F6118883A88220F507F65F
:050CF000A883758300DC
:010CF50022DC
:030CF600F280F792
:020CF900F022E7
:080095007800E84400600A79DC
:03009D000075A04B
:0600A00000E4F309D8FCA6
:0800A60078E1E84400600C79E8
:0B00AE0001900001E4F0A3D8FCD9FA97
:030CFB00120330B1
:090CFE007900E583B58202800D46
:050D07005003121ABDAB
:080D0C00E583C3958212229ECB
:080D1400E5D0C465D020E11711
:0E0D1C00EA2DFAEB3EFBEC3FFC50097401128D
:060D2A00229EEC4480FC57
:030D30000211D6D7
:0E0D3300C3EA9DFAEB9EFBEC9FFC500FC3E45D
:0D0D410099F9E49AFAE49BFBE49CFCB2D122
:060D4E0012035E0211D643
:0200BB00D2066B
:0C0D5400A2AF9204C2AF43A220A982907B
:0E0D60000056E0FA900057E0FB8A838B821267
:0C0D6E00FFF0F58253A2DFA20492AF2236
:0A0D7A00200607E4A2053324FF223F
:080D8400C206900056E4F09055
:0E0D8C0000577403F0758200120D54AA82E421
:040D9A00BA80010416
:0A0D9E0024FF9205E4A2053324FFB0
:010DA8002228
:0D0DA90090000F12025D758203122235903A
:0E0DB600000512025D7582031222357582035C
:0D0DC400122235758203122235758220122D
:0C0DD100226375820112226375820C12ED
:080DDD0022637582010222630A
:0E0DE500E58290007BF090007BE0FA6005BA9A
:040DF300011E800E4F
:0E0DF70090007AE0FA74802AFAF582022263F4
:0E0E050090007AE0FA74C02AFAF582022263A5
:010E130022BC
:0E0E1400E58290007FF090007FE0FAC4035466
:0E0E2200F8FA74402AFAF58212226390007CDE
:0A0E3000E0FAA3E0FBA3E0FC7D085C
:0E0E3A008A828B838CF01221AEFEA3AA82ABBB
:0E0E4800838E82C002C003C004C00512220DBA
:0B0E5600D005D004D003D002DDDA226A
:040E61007A017B0097
:0E0E6500C3EA9402EB6480948050558A041C0A
:0A0E7300ECC454F0245AFCE43400EF
:0E0E7D00FD7E008A07EBC454F0CFC4CF6FCFC8
:0B0E8B0054F0CF6FF8EF245AFFE8345A
:0C0E960000F8900087EFF0A3E8F0A374D0
:0E0EA20000F090008A7410F0E4A3F08C828DB2
:0E0EB000838EF0C002C003121108D003D002DE
:070EBE000ABA00A30B80A09B
:0E0EC50090008F7420F09000907410F0E4A361
:0A0ED300F090006A75F00002117E35
:040EDD007A007B001C
:0E0EE100C3EA9402EB6480948050718A0490FE
:0E0EEF00007AE4F08C82C002C003120DE5D040
:0E0EFD0003D0028A04EBC454F0CCC4CC6CCCFD
:090F0B0054F0CC6CFD7E007F0067
:0D0F1400C3EE9410EF648094805036EC24FE
:0A0F21005AF8ED3400F9EE28F582CD
:0E0F2B00EF39F583E0F8F582C002C003C00480
:0E0F3900C005C006C00712220DD007D006D09A
:0E0F470005D004D003D0020EBE00C20F80BF42
:050F55000ABA00010BC7
:030F5A00020EE1A3
:010F5D002271
:0A0F5E0075820C122263120EDD9062
:0A0F68000058E0FA900059E0FB90F9
:0C0F7200007AF08A82120DE575820D02F3
:020F7E002263EC
:0D0F8000900058E0FA90005874012AF0909B
:0E0F8D000058E0FAC3648094824009120E619D
:060F9B009000587401F003
:010FA100222D
:0E0FA200E582900080F0900058E0FAC454F010
:080FB000245AFAE43400FB901E
:0E0FB8000059E0FC2AFAE43BFB900080E0FDCB
:0D0FC6008A828B83F090005974012CF0900A
:0E0FD3000059E0FAC3648094904008900059E1
:050FE100E4F0020F80A6
:010FE60022E8
:0E0FE700E582900081F0900081E0FABA0902E4
:020FF500801664
:050FF700BA0A028009A6
:090FFC00BA0D26900059E4F02220
:08100500900059E4F0020F8095
:0E100D00758220120FA2758220120FA275822A
:0A101B0020120FA2758220020FA21E
:051025008A82020FA207
:07102A0012025A120DA990F9
:091031000058E4F0900059F09021
:0E103A00008F7420F09000907420F0E4A3F07A
:0A10480090005A75F00012117E02AC
:021052000F5E2F
:08105400AA82120FE7020F5EF1
:0E105C00AAF0AB83E582900082F0A3EBF0A334
:0E106A00EAF0900082E0FAA3E0FBA3E0FC7D38
:03107800007E00F7
:0E107B00ED2AFFEE3BF88C018F82888389F00E
:0E1089001221AEFF60208F82C002C003C0049F
:0E109700C005C006120FE7D006D005D004D069
:0A10A50003D0020DBD00CF0E80CC79
:0310AF00020F5ECF
:0C10B200E582900086F0900086E0FA9045
:0910BE000058F0900085E0FB9061
:0B10C7000059F090007AEBF08A8202E2
:0210D2000DE52A
:0E10D40090008F7420F09000907420F0E4A340
:0E10E200F090005A75F00012117E7582011216
:0B10F0002263900085E4F0758200028E
:0210FB0010B231
:01235A001072
:01235B00027F
:0B10FD007F8E1222E3F58385F0822233
:0E110800AAF0AB83E58290008CF0A3EBF0A37D
:0B111600EAF090008CE0F517A3E0F574
:0611210018A3E0F519908F
:0C1127000087E0FDA3E0FEA3E0FF8517B9
:0311330014851808
:0311360015851903
:091139001690008AE0F8A3E0F929
:091142008802890318B8FF0119A5
:0E114B00EA4B60258D828E838FF01221AEFA62
:0A115900A3AD82AE838514828515D4
:0B116300838516F0EA120CE2A38582DF
:06116E001485831580CEFC
:0711740085178285188385B1
:03117B0019F02246
:0E117E00AAF0AB83E582900092F0A3EBF0A301
:0E118C00EAF0900092E0FAA3E0FBA3E0FC90F2
:0C119A00008FE0FD900090E0FEA3E0FF5D
:0911A6008E008F011EBEFF011F27
:0E11AF00E84960118A828B838CF0ED120CE20D
:0711BD00A3AA82AB8380E2CC
:0E11C400900092E0FAA3E0FBA3E0FC8A828B8D
:0411D200838CF022F8
:0611D600B98003EA13B327
:0E11DC004010EA2401FAE43BFBE43CFC500422
:0411EA007C8005827E
:0911EE00BC000EBB000BBA0008A6
:0811F700E4F5F0F583F5822216
:0E11FF00A2D1E582138CF092F78B838A8222B4
:0D120D00E4F583F58275F080F4A2D1132280
:0B121A00E4F583F58275F0C0747F22BC
:08122500C00E85810EAA8212A1
:05122D0000C7D00E22F5
:0E123200AAF0AB83E582900096F0A3EBF0A348
:0E124000EAF0900096E0FAA3E0FBA3E0FC9039
:0E124E000095E0FD9000A9E4F0A3F0A3F0905D
:0E125C0000ACEAF0A3EBF0A3ECF09000AFEDD5
:07126A00F090122502138A27
:06127100C00E85810EE5B0
:0C1277000E24FBFA9000A9E4F0A3F0A301
:0C128300F0E50E24FBF89000ACE6F0084B
:0D128F00A3E6F008A3E6F09000AFEAF090AF
:0A129C00122512138AAA82AB83D038
:0212A6000E2216
:0C12A800E5829000A5F09000A5E0FA900F
:0E12B400009BE0C0E0A3E0C0E0A3E0C0E07457
:0812C200D6C0E07412C0E090F8
:0C12CA000099E0C0E0A3E0C0E08A8222AE
:0E12D6001581158115819000A3E0FAA3E0FBBD
:0C12E4009000A374012AF0E43BA3F02268
:0E12F000E5829000A6F09000A6E0FA74302A85
:0C12FE00FA24C6500A74072AFA300703CD
:03130A004302207B
:05130D008A820212A813
:0E131200E5829000A7F09000A7E0FAC4540F07
:0E132000FBF582C0021212F0D00253020F8AB7
:04132E00820212F035
:0E133200E5829000A8F090009EE0FAA3E0FB98
:0E134000A3E0FCA3E0FD9000A2E0FE9000A858
:04134E00E0FF782024
:0E135200EE2EFEED235401F94206EA2AFAEBD4
:0E13600033FBEC33FCED33FDC3EE9F4007EE94
:06136E00C39FFE430201D3
:0E137400D8DC90009EEAF0A3EBF0A3ECF0A30F
:08138200EDF09000A2EEF02254
:0E138A00AA83E5829000B0F0A3EAF09000B0D4
:0E139800E0FAA3E0FB900099EAF0A3EBF090DE
:0E13A60000A9E0FAA3E0FBA3E0FC90009BEAA4
:0E13B400F0A3EBF0A3ECF09000A3E4F0A3F0A4
:0E13C2009000ACE0FAA3E0FBA3E0FC8A828B73
:0E13D000838CF01221AEFD9000AC74012AF067
:0D13DE00E43BA3F0A3ECF0ED7003021AB1A4
:0513EB00BD2502800396
:0313F000021AA935
:0513F300C208C209C29E
:0413F8000AC20BC258
:0413FC000CC20DC250
:041400000EC20F9079
:0914040000B2E4F09000B3F09096
:0E140D0000B474FFF09000ACE0FAA3E0FBA383
:02141B00E0FCF3
:0E141D008A828B838CF01221AEFEA3AA82ABD2
:0D142B00839000ACEAF0A3EBF0A3ECF0908E
:0D14380000B6EEF0BE25088E821212A8024A
:0214450013C2D0
:051447008E07BF30001C
:0E144C0040498E07EF24C640429000B4E0FFF6
:0E145A00BFFF29C002C003C0049000B3E0FA37
:0E14680075F00AA4FAEE24D09000B32AF0909A
:0D14760000B3E0FAD004D003D002709BD286
:0314830009809746
:0E148600EF75F00AA4FFEE24D09000B42FF012
:0314940002141D22
:0E1497009000B6E0FEBE2E089000B4E4F00215
:0214A500141D14
:0E14A7008E82C002C003C004C006122308E5F6
:0C14B5008224FF9207D006D004D003D0A0
:0B14C100023007079000B674DF5EF0F9
:0A14CC009000B6E0FEBE200280553D
:0514D600BE2B02804B5B
:0514DB00BE2D0280415E
:0514E000BE4202804B3A
:0514E500BE430280502F
:0614EA00BE440302171EC0
:0614F000BE460302174096
:0614F600BE490302171EAF
:0514FC00BE4C0280342B
:06150100BE4F0302172893
:06150700BE500302168035
:05150D00BE5302804204
:06151200BE550302173074
:06151800BE580302173863
:03151E000217446D
:05152100D20802141DB8
:05152600D20A02141DB1
:05152B00D20B02141DAB
:05153000D20D02141DA4
:05153500D20E02141D9E
:0E153A009000AFE0FA24FEF89000AFF08602B9
:0C154800088603188A821212A8021750AD
:0E1554009000AFE0FA24FDF89000AFF08602A0
:0E156200088603088604181890009EEAF0A37D
:0E157000EBF0A3ECF090009EE0FAA3E0FBA3EA
:0E157E00E0FC8A828B838CF0121CE4AA82AB04
:0E158C00839000B4E0FBBBFF059000B4EAF0D2
:0C159A002008389000B3E0FBC3EA9B502F
:0D15A6002E9000B3EBC39AF09000B3E0FB71
:0D15B3008B041B9000B3EBF0BC0002801015
:0E15C000758220C002C0031212A8D003D00210
:0215CE0080E3B8
:0515D0009000B3EBF0F8
:0515D5009000B4E0FDF0
:0E15DA00C00290009EE0FCA3E0FFA3E0FA8CAC
:0E15E800828F838AF01221AED00260538D04F0
:0E15F6001DC374808CF063F08095F05044C0EB
:0A1604000290009EE0F50FA3E0F550
:08160E0010A3E0F511740125A1
:071616000FFBE43510FAACF4
:0C161D001190009EEBF0A3EAF0A3ECF0AB
:07162900850F828510838507
:0C16300011F01221AEFAF582C002C005D4
:0B163C001212A8D005D002D00280934B
:0616470020080302175009
:0D164D009000B3E0FBC3EA9B40030217507E
:0C165A009000B3EBC39AF09000B3E0FAEC
:0E1666008A031A9000B3EAF0BB000302174B90
:0C167400758220C0021212A8D00280E68D
:0E1680009000AFE0FB24FDF89000AFF0860371
:0E168E00088604088607181890009EEBF0A34B
:0E169C00ECF0A3EFF09000A0E0FB247F5008DC
:0816AA009000B67443F08020AB
:0D16B200EB249F50089000B67450F0801398
:0D16BF00EB24BF50089000B67449F080067F
:0616CC009000B67458F016
:0E16D2009000B6E0FBF582C0031212A8D00310
:0E16E00075823AC0031212A8D003758230C082
:0E16EE00031212A8D003758278C0031212A84E
:0716FC00D003BB4902800F7F
:05170300BB5002800A4A
:0A17080090009FE0FBF5821213121F
:0C17120090009EE0FBF582121312803262
:0A171E00D20C9000B2740AF080288B
:081728009000B27408F080206B
:081730009000B2740AF0801869
:081738009000B27410F0801063
:04174000D20F800C38
:071744008E821212A880053D
:05174B009000B3EAF07C
:0C175000300F6B9000AFE0FA24FCF89022
:0E175C0000AFF08602088603088604088606A1
:0E176A0018181890009EEAF0A3EBF0A3ECF024
:0B177800A3EEF090009E745CF0A374E0
:0617830023F0A37480F0C6
:0E17890090009EE0FBA3E0FCA3E0FD74012BAA
:0E179700FEE43CFF8D0290009EEEF0A3EFF00A
:0E17A500A3EAF08B828C838DF01221AEFA70D5
:0417B300030213C258
:0717B7008A821212A880CB08
:0B17BE009000B2E0FABA00030213C270
:0817C9009000BD74BCF0A37494
:0617D10000F0300D4C9009
:0E17D70000AFE0FA14F89000AFF08602EA339B
:0E17E50095E0FBFCFE90009EEAF0A3EBF0A363
:0B17F300ECF0A3EEF0300C030218989D
:0E17FE0090009EE0FAA3E0FBA3E0FCA3E0FE57
:0E180C007B007C007E0090009EEAF0A3EBF0D3
:08181A00A3ECF0A3EEF08076D0
:0C182200300E2A9000AFE0FA24FCF89091
:0E182E0000AFF08602088603088604088606CE
:0E183C0018181890009EEAF0A3EBF0A3ECF051
:05184A00A3EEF080494F
:0E184F009000AFE0FA24FEF89000AFF08602A1
:0E185D0008860318EB3395E0FCFE90009EEA2F
:0C186B00F0A3EBF0A3ECF0A3EEF0200CD7
:0E1877002090009EE0FAA3E0FBA3E0FCA3E0BB
:0E188500FE7C007E0090009EEAF0A3EBF0A334
:05189300ECF0A3EEF0F3
:0C189800300C3E90009EE0FAA3E0FBA3A1
:0E18A400E0FCA3E0FE30E72B90009EE0FAA3EC
:0E18B200E0FBA3E0FCA3E0FEC3E49AFAE49B93
:0E18C000FBE49CFCE49EFE90009EEAF0A3EB8D
:0918CE00F0A3ECF0A3EEF080029F
:0218D700C20C41
:0818D900D2109000B2E0FC7592
:0318E10012BC75C1
:0418E40013007D0070
:0E18E8009000A2E4F08C82C004C005121332FE
:0C18F600D005D004201032C0049000A2E5
:0A190200E0FFC4FF85128285138305
:0A190C00E0FA42078512828513837A
:0A191600EFF0151274FFB512021570
:0119200013B3
:081921009000BDE512F0A3E502
:0619290013F0D004800C55
:09192F009000A2E0FF8512828500
:031938001383F026
:09193B000D9000B5EDF0B2109022
:0E194400009EE0FFA3E0FAA3E0FEA3E0FBEFAD
:0C1952004A4E4B70919000BDE512F0A3CE
:09195E00E513F09000B5EDF090E6
:0C19670000B3E0FA70069000B37401F0C9
:0A19730020092720082474012DFA32
:05197D009000B3E0FB47
:0D198200C3EA9B5011758220C002C0031201
:09198F0012A8D003D0021B80EA6B
:051998009000B3EBF02C
:0A199D00300C1275822D1212A89072
:0B19A70000B3E0FA149000B3F0802FB2
:0C19B2009000B5E0FA6028300A1275823F
:0B19BE002B1212A89000B3E0FA149066
:0519C90000B3F08013E3
:0A19CE00300B107582201212A89051
:0919D80000B3E0FA149000B3F032
:0919E10020082F9000B5E0FA90F7
:0419EA0000B3E0FB6B
:0E19EE008B041B9000B3EBF0C3EA9C50363024
:0619FC0009047C308002AA
:021A02007C2046
:0E1A04008C82C002C0031212A8D003D0028050
:011A1200DBF8
:0E1A13009000B3E0FA9000B5E0FCC39A5009D1
:091A21009000B3EAC39CF0800CB4
:071A2A009000B3E4F0800519
:051A31009000B3EBF092
:0D1A36009000BDE0FAA3E0FB9000B5E0FCDD
:0A1A43008C061CEE6040B21020106B
:061A4D00150ABA00010BAE
:0E1A53008A828B83E0FEC4540FFE9000A2F046
:021A6100800EF5
:0E1A63008A828B83E0FE53060F9000A2EEF005
:0E1A71009000A2E0FEF582C002C003C0041285
:0A1A7F0012F0D004D003D00280BAA8
:061A89002008030213C255
:051A8F009000B3E0FA35
:091A94008A031AEB70030213C26D
:0C1A9D00758220C0021212A8D00280EB5B
:081AA9008D821212A80213C283
:0C1AB1009000A3E0FAA3E08A82F58322F3
:0B235C003C4E4F20464C4F41543E00C9
:0E1ABD00E582C583F582A2D133A2D592D11362
:0C1ACB0092D5ECCFFCEBCEFBEACDFA226A
:0B1AD700E5829000C1F0301102C294C3
:091AE2009000C1E0FA7B007C00D9
:0E1AEB008A057E009000D07488F0A37413F07A
:0E1AF9008D828E83C002C003C004121CC4ADD7
:0E1B070082AE83D004D003D002C3EB9DEC6409
:0E1B1500808EF063F08095F050070BBB00C887
:031B23000C80C56E
:051B2600301102D29411
:011B2B002297
:0C1B2C00E582FA90236793FAC4540FFB83
:021B38007C002F
:0D1B3A00C3EC9B50528CF005F0740180024A
:021B470025E097
:0C1B4900D5F0FBFD5A6016D21175820326
:0E1B5500C002C003C004121AD7D004D003D0BF
:031B6300028014E9
:0C1B6600D211758201C002C003C004123D
:081B72001AD7D004D003D00201
:0C1B7A00C211758201C002C003C0041239
:0B1B86001AD7D004D003D0020C80A9B5
:0C1B9100C211758203C002C003121AD7F3
:061B9D00D003D002809588
:0A1BA300121DFA900014121DFBC27F
:0A1BAD0013900014121E18D2949039
:051BB7001B2C021BDDE8
:0C1BBC00E5829000C2F09000C2E0FA74D4
:081BC800DCC0E0741BC0E090DA
:0C1BD00000BFE0C0E0A3E0C0E08A822279
:011BDC0022E6
:0E1BDD00AA83E5829000C3F0A3EAF09000C353
:0E1BEB00E0FAA3E0FB9000BFEAF0A3EBF022CB
:0E1BF900E5829000C5F09000C5E025E0FA24DA
:0A1C0700E5F582E43400F583E0FA0D
:0C1C1100A3E0FB7C808A828B838CF02295
:032367000021480A
:09236A004E6F206572726F720063
:0E23730049324320646576696365206E6F749D
:092381002070726573656E740032
:0E238A004932432064657669636520646964A6
:09239800206E6F742061636B007C
:0223AC006A23A2
:0223AE00732397
:0223B0008A237E
:0200BD00C2126D
:0E1C1D00C2AF9000C6E0FAA3E0FBA3E0FCA378
:0E1C2B00E0FD9000CAEAF0A3EBF0A3ECF0A3FA
:0C1C3900EDF0D2AF8A828B838CF0ED229C
:0E1C4500C0E0C082C083C0D075D0009000C641
:0E1C5300E02401F0A3E03400F0A3E03400F040
:0E1C6100A3E03400F0C2CFD0D0D083D082D028
:021C6F00E03261
:041C7100301201220A
:0E1C750075C900C2C9C2C8C2CDC2CCC2CBC2A2
:0D1C8300CAC2CF120D7AE433FABA010E90F6
:0D1C900000CE74F3F09000CF74FFF0800CD4
:0C1C9D009000CE74F9F09000CF74FFF0BE
:0E1CA9009000CEE0FA8ACD9000CFE0FB8BCC0D
:0C1CB7008ACB8BCAD2CAD2AFD2E8D212BC
:011CC30022FE
:0E1CC400AA83AB828BF09000D0E0A4F8A9F0C8
:0E1CD2008AF0E0A429F98BF0A3E0A429F583A1
:041CE00088822222B2
:0E1CE400AAF0AB83E5829000D2F0A3EBF0A350
:0E1CF200EAF07A007B009000D2E0FCA3E0FD57
:031D0000A3E0FE5F
:0E1D03008C828D838EF01221AEFFA3AC82ADD8
:0E1D1100839000D2ECF0A3EDF0A3EEF0EF60B3
:081D1F00070ABA00DF0B80DCAB
:0E1D27009000D2ECF0A3EDF0A3EEF08A828BD8
:021D3500832207
:081D370012033030D502B2D1D5
:091D3F00BF0009BC000302121AE6
:031D480002120D77
:061D4B00BC00030211F7C9
:0D1D5100E583B4FF0BE582B4FF0302121A14
:031D5E000211F778
:081D6100E582B4FF0302120D3C
:0C1D6900C395835007247F400B0211F744
:081D7500248014500302120D3A
:0E1D7D00F582C3ED9AEE9BEF9C40111582C3D8
:0E1D8B00EA33F9EB33FAEC33FBE433FC80056A
:051D9900E4CCCBCAF907
:051D9E00C08275F01980
:0E1DA300C3E99DEA9EEB9FEC9400D5F0028010
:011DB1002D04
:0E1DB200400EE99DF9EA9EFAEB9FFBEC9400CF
:021DC000FCC362
:0E1DC200B3E833F8E58233F582E58333F58329
:0E1DD000C3E933F9EA33FAEB33FBEC33FC8062
:011DDE00C440
:0E1DDF00B3E4F938FAE43582FBE43583FCD036
:071DED0082500405827C8096
:061DF40012035E0211EE75
:011DFA0022C6
:011DFB0022C5
:0E1DFC00AA83E5829000D5F0A3EAF09000D50E
:0C1E0A00E0FAA3E0FBD2148A828B830272
:021E16001E3676
:0E1E1800AA83E5829000D7F0A3EAF09000D7ED
:0A1E2600E0FAA3E0FBA21392148A75
:061E3000828B83021E36C6
:0E1E3600AA83E5829000D9F0A3EAF09000D9CB
:091E4400E0FAA3E0FB30E7012203
:0E1E4D00C374439A74808BF063F08095F0505C
:021E5B00012262
:0D1E5D00EA240983C0E0EA244783C0E022A4
:021E6A00F2F78D
:021E6C00FC0177
:021E6E00060B61
:021E700010154B
:021E7200BDBDF4
:021E7400BDBDF2
:021E7600BDBDF0
:021E7800BDBDEE
:021E7A001A1F2D
:021E7C00242917
:021E7E002E3301
:021E8000383DEB
:021E8200BDBDE4
:021E8400BDBDE2
:021E8600BDBDE0
:021E8800BDBDDE
:021E8A004247CD
:021E8C004C51B7
:021E8E00565BA1
:021E900060658B
:021E9200BDBDD4
:021E9400BDBDD2
:021E9600BDBDD0
:021E9800BDBDCE
:021E9A006A6F6D
:021E9C00747957
:021E9E007E8341
:021EA000888D2B
:021EA200BDBDC4
:021EA400BDBDC2
:021EA600BDBDC0
:021EA800BDBDBE
:021EAA00929D07
:021EAC00A8B3D9
:021EAE001E1EF6
:021EB0001E1FF3
:021EB2001F1FF0
:021EB4001F1FEE
:021EB6001F1FEC
:021EB8001F1FEA
:021EBA001F1FE8
:021EBC001F1FE6
:021EBE001F1FE4
:021EC0001F1FE2
:021EC2001F1FE0
:021EC4001F1FDE
:021EC6001F1FDC
:021EC8001F1FDA
:021ECA001F1FD8
:021ECC001F1FD6
:021ECE001F1FD4
:021ED0001F1FD2
:021ED2001F1FD0
:021ED4001F1FCE
:021ED6001F1FCC
:021ED8001F1FCA
:021EDA001F1FC8
:021EDC001F1FC6
:021EDE001F1FC4
:021EE0001F1FC2
:021EE2001F1FC0
:021EE4001F1FBE
:021EE6001F1FBC
:021EE8001F1FBA
:021EEA001F1FB8
:021EEC001F1FB6
:021EEE001F1FB4
:021EF0001F1FB2
:051EF200A21492802201
:051EF700A214928122FB
:051EFC00A214928222F5
:051F0100A214928322EE
:051F0600A214928422E8
:051F0B00A214928522E2
:051F1000A214928622DC
:051F1500A214928722D6
:051F1A00A214929022C8
:051F1F00A214929122C2
:051F2400A214929222BC
:051F2900A214929322B6
:051F2E00A214929422B0
:051F3300A214929522AA
:051F3800A214929622A4
:051F3D00A2149297229E
:051F4200A21492A02290
:051F4700A21492A1228A
:051F4C00A21492A22284
:051F5100A21492A3227E
:051F5600A21492A42278
:051F5B00A21492A52272
:051F6000A21492A6226C
:051F6500A21492A72266
:051F6A00A21492B02258
:051F6F00A21492B12252
:051F7400A21492B2224C
:051F7900A21492B32246
:051F7E00A21492B42240
:051F8300A21492B5223A
:051F8800A21492B62234
:051F8D00A21492B7222E
:071F920030140443A10122F9
:041F990053A1FE2230
:071F9D0030140443A10222ED
:041FA40053A1FD2226
:071FA80030140443A10422E0
:041FAF0053A1FB221D
:071FB30030140443A10822D1
:031FBA0053A1F739
:011FBD002201
:0E1FBE00AA83E5829000DBF0A3EAF09000DB3E
:0B1FCC00E0FAA3E0FB30E70302219ADB
:0E1FD700C374439A74808BF063F08095F050D1
:041FE5000302219A38
:0D1FE900EA240983C0E0EA244783C0E02217
:021FF6007E85E6
:021FF8008C93C8
:021FFA009AA1AA
:021FFC00A8AF8C
:021FFE009A9AAD
:022000009A9AAA
:022002009A9AA8
:022004009A9AA6
:02200600B6BD65
:02200800C4CB47
:02200A00D2D929
:02200C00E0E70B
:02200E009A9A9C
:022010009A9A9A
:022012009A9A98
:022014009A9A96
:02201600EEF5E5
:02201800FC03C7
:02201A000A11A9
:02201C00181F8B
:02201E009A9A8C
:022020009A9A8A
:022022009A9A88
:022024009A9A86
:02202600262D65
:02202800343B47
:02202A00424929
:02202C0050570B
:02202E009A9A7C
:022030009A9A7A
:022032009A9A78
:022034009A9A76
:022036005E6DDD
:022038007C8B9F
:02203A00202064
:02203C00202062
:02203E00202060
:0220400020205E
:0220420021215A
:02204400212158
:02204600212156
:02204800212154
:02204A00202054
:02204C00202052
:02204E00202050
:0220500020204E
:0220520021214A
:02205400212148
:02205600212146
:02205800212144
:02205A00202044
:02205C00202141
:02205E0021213E
:0220600021213C
:0220620021213A
:02206400212138
:02206600212136
:02206800212134
:02206A00212132
:02206C00212130
:02206E0021212E
:0220700021212C
:0220720021212A
:02207400212128
:02207600212126
:02207800212124
:02207A00212122
:02207C00212120
:07207E00E4A2803324FF22DD
:07208500E4A2813324FF22D5
:07208C00E4A2823324FF22CD
:07209300E4A2833324FF22C5
:07209A00E4A2843324FF22BD
:0720A100E4A2853324FF22B5
:0720A800E4A2863324FF22AD
:0720AF00E4A2873324FF22A5
:0720B600E4A2903324FF2295
:0720BD00E4A2913324FF228D
:0720C400E4A2923324FF2285
:0720CB00E4A2933324FF227D
:0720D200E4A2943324FF2275
:0720D900E4A2953324FF226D
:0720E000E4A2963324FF2265
:0720E700E4A2973324FF225D
:0720EE00E4A2A03324FF224D
:0720F500E4A2A13324FF2245
:0720FC00E4A2A23324FF223D
:07210300E4A2A33324FF2234
:07210A00E4A2A43324FF222C
:07211100E4A2A53324FF2224
:07211800E4A2A63324FF221C
:07211F00E4A2A73324FF2214
:07212600E4A2B03324FF2204
:07212D00E4A2B13324FF22FC
:07213400E4A2B23324FF22F4
:07213B00E4A2B33324FF22EC
:07214200E4A2B43324FF22E4
:07214900E4A2B53324FF22DC
:07215000E4A2B63324FF22D4
:07215700E4A2B73324FF22CC
:09215E00E5A130E0047A018002E1
:022167007A00FC
:04216900EA24FF2243
:09216D00E5A130E1047A018002D1
:022176007A00ED
:04217800EA24FF2234
:09217C00E5A130E2047A018002C1
:022185007A00DE
:04218700EA24FF2225
:09218B00E5A130E3047A018002B1
:022194007A00CF
:04219600EA24FF2216
:04219A00E424FF2218
:03003F00758122A6
:0A00420012219EE58260030200C255
:07219E00758E009000002285
:0921A50012003E121BA3C2A62287
:0823A10024002500260027009E
:0E21AE0020F71430F6148883A88220F507E687
:0621BC00A88375830022D8
:0321C200E280F7C1
:0321C500E493227E
:0221C800E02213
:0B21CA00E4AC82FBFAF9748602229458
:0A21D50090000112025DE424FF22D5
:0D21DF00E5829000DDF0C2A5D2A4D2A6904A
:0D21EC0000DDE0FAC454F0FA9000DDF09040
:0E21F90000DDE0FA74F05A428043020FEA5211
:0622070080C2A6D2A52250
:06220D00E5829000DEF006
:0E2213001221D540FB9000DEE0FAC4540FFB10
:0E22210053030F8B82C0021221DFD002530242
:06222F000F8A820221DF8C
:0D223500E5829000DFF0C2A5C2A4D2A69001
:0D22420000DFE0FAC454F0FA9000DFF090E5
:0E224F0000DFE0FA74F05A428043020FEA52B8
:06225D0080C2A6D2A522FA
:06226300E5829000E0F0AE
:0E2269001221D540FB9000E0E0FAC4540FFBB8
:0E22770053030F8B82C002122235D002530295
:062285000F8A82022235DF
:09228B00FCABF0AA83A982749E49
:02229400C2D1B5
:08229600F58212035E0211D66D
:09229E006040F82582500274FF33
:0E22A700F582E824F8501ECCCBCAF9E4CC2412
:0E22B500F85014CBCAF9E4CB24F8500BCAF948
:0922C300E4CA24F850037900225A
:0522CC0024086010F879
:0E22D100C3EC13FCEB13FBEA13FAE913F9D884
:0122DF00F10D
:0122E00022DB
:0222E1007F9EDE
:0922E30012232530D1030211F78A
:0E22EC00C3EF9582500974FFF5F0F583F5827B
:0122FA0022C1
:0522FB00790012229E93
:0823000089828A838BF0EC2234
:0E230800E5829000E1F09000E1E0FABA610099
:0B2316004009EA248540047582012282
:04232100758200229F
:01003E00229F
:08006E007909E94400601A7AE7
:050076000143A201900E
:05007B0023A915A2906D
:0800800000E2E405A293A315C0
:07008800A2F0A3D9F5DAF3A1
:0D232500AA82AB83A2F73392D16002D2F7F7
:05233200F582ACF02271
:00000001FF
